:1000000000008A150A12642FF200030E8301F1002A
:100010000A088A01F000040883160317D00083162B
:100020000317CB01831203130B1D19288316031723
:10003000CB0A831603174B08013A031D24288A159F
:100040000A1273218A110A128316031750088400BA
:1000500070088A008301710E8300F20E720E09008F
:1000600083160313A3007F08A2007E08A1007D0869
:1000700083160313B30083160313A0007C08A700A4
:100080007B08A6007A08A500790883160313B70039
:1000900083160313A400210883160313B4008316E8
:1000A0000313220883160313B500831603132308D2
:1000B00083160313B6008316031325088316031350
:1000C000B80083160313260883160313B90083169A
:1000D0000313270883160313BA0083160313330888
:1000E00083160313A0008316031334088316031327
:1000F000A10083160313350883160313A200831689
:100100000313360883160313A300200821042204D6
:1001100023040319A928831603133708831603132E
:10012000A00083160313380883160313A100831657
:100130000313390883160313A200831603133A0826
:1001400083160313A3002008210422042304031DA3
:10015000B1280030FD000030FE000030FF0000300C
:10016000CC2B83160313330883160313A0008316C6
:100170000313340883160313A100831603133508F1
:1001800083160313A2008316031336088316031382
:10019000A300230DA401A40DA501A601A701013010
:1001A0002405A000A101A201A301831603133708AF
:1001B00083160313A400831603133808831603134E
:1001C000A50083160313390883160313A6008316AC
:1001D00003133A0883160313A700270DA801A80DDF
:1001E000A901AA01AB0101302805A400A501A601BF
:1001F000A7012408A0060030A1060030A2060030A6
:10020000A3062008A40083160313330883160313E0
:10021000A00083160313340883160313A10083166A
:100220000313350883160313A2008316031336083D
:1002300083160313A300220D230DA000A500A60121
:10024000A60DA701A801A101A201A3018230A00768
:10025000FF30031CA107FF30031CA207FF30031C63
:10026000A3072008A5002108A6008316031337085A
:1002700083160313A0008316031338088316031391
:10028000A10083160313390883160313A2008316F3
:1002900003133A0883160313A300220D230DA000B5
:1002A000A700A801A80DA901AA01A101A201A3010B
:1002B0002508A7002608A8000030A81BFF30AA00C8
:1002C000A90020082707A00028080318280FA10765
:1002D00029080318290FA2072A0803182A0FA307C1
:1002E0002008A5002108A6008316031333088316EF
:1002F0000313A00083160313340883160313A1000D
:1003000083160313350883160313A2008316031301
:10031000360883160313A300A213A301A217200813
:1003200083160313B30083160313210883160313E4
:10033000B40083160313220883160313B50000309C
:10034000B60083160313370883160313A000831621
:100350000313380883160313A10083160313390807
:1003600083160313A200831603133A08831603139C
:10037000A300A213A301A217200883160313B7003A
:1003800083160313210883160313B800831603137F
:10039000220883160313B9000030BA008316031332
:1003A000330883160313A00083160313340883163F
:1003B0000313A700A1008316031335088316031344
:1003C000A800A20083160313360883160313A9009E
:1003D000A300AA0183160313370883160313A00092
:1003E00083160313380883160313AB00A10083168A
:1003F0000313390883160313AC00A20083160313FA
:100400003A0883160313AD00A300AE012B08F900D0
:100410002C08FA002D08FB000030FC002708FD0026
:100420002808FE002908FF0000308A110A16002063
:100430008A110A1283160313A3007F08A2007E0804
:10044000A1007D08A000831603133308831603134D
:10045000A70083160313340883160313A80083161A
:100460000313350883160313A900831603133608F4
:1004700083160313AA00A801A901AA018316031376
:10048000370883160313AB0083160313380883164B
:100490000313AF00AC00831603133908831603134C
:1004A000AD00831603133A0883160313AE00B2019E
:1004B0002F08F9002D08B000FA002E08B100FB004B
:1004C0000030FC002708FD000030FE000030FF0077
:1004D00000308A110A1600208A110A1283160313AB
:1004E000AD00AA007F08AC00A9007E08AB00A80000
:1004F0007D08A700AE012B08A0072C0803182C0FBD
:10050000A1072D0803182D0FA2072E0803182E0F80
:10051000A30783160313370883160313A700831654
:100520000313380883160313A8008316031339082E
:1005300083160313A900831603133A0883160313C3
:10054000AA00A801A901AA01831603133308831680
:100550000313AB0083160313340883160313AC0094
:1005600083160313350883160313B000AD008316FA
:100570000313360883160313B100AE00B2012C0832
:10058000AF00F9003008FA003108FB000030FC0031
:100590002708FD000030FE000030FF0000308A1107
:1005A0000A1600208A110A1283160313AD00AA004E
:1005B0007F08AC00A9007E08A8007D08A700AE0156
:1005C0002808AB00A00703182C0FA1072D0803185B
:1005D0002D0FA2072E0803182E0FA307A7018030A6
:1005E0002305AA002A080319052B8030A007031849
:1005F000A10A0319A20A0319A30A2108A0002208CC
:10060000A1002308A200A3011C2B40308316031372
:10061000A0070318A10A0319A20A0319A30A200DAF
:10062000210DA000220DA100230DA200A301A30D06
:10063000FF30A507031CA60383160313A213260885
:10064000803E7F3E031D262B00302502031C552BC8
:100650008316031324080319332BA701A801A9014A
:100660008030AA00392B83160313A701A801A90122
:10067000AA0183160313A9177F30AA04270883163B
:100680000313B30083160313280883160313B4005F
:1006900083160313290883160313B5008316031367
:1006A0002A0883160313B600AD2B03148316031315
:1006B000A61F0310031C632B83160313B301B4019D
:1006C000B501B601AD2B00308316031324040319C2
:1006D0006F2BA401A701A8018030A900752B8316F8
:1006E0000313A401A701A801A90183160313250878
:1006F000AA002608AB000030AB1BFF30AD00AC00F9
:100700002B0C2A0CAF00AE01AE0CA601A5010030E7
:10071000A4040030A7042E08A8042F08A904240864
:10072000A0042708A1042808A2042908A30420087B
:1007300083160313B30083160313210883160313D0
:10074000B40083160313220883160313B50083161F
:100750000313230883160313B60083160313330809
:1007600083160313A00083160313340883160313A0
:10077000A10083160313350883160313A200831602
:100780000313360883160313A3002008FD00210875
:10079000FE002208FF002308080083120313A300B1
:1007A0007F08A2007E08A1007D0883120313BB000E
:1007B00083120313A0007C08A7007B08A6007A0818
:1007C000A500790883120313BF0083120313A4004A
:1007D000A801A901AA01AB01210883120313BC00DF
:1007E00083120313220883120313BD008312031321
:1007F000230883120313BE008312031325088312F8
:100800000313C00083120313260883120313C100CD
:1008100083120313270883120313C20083120313E6
:100820003B0883120313A000831203133C088312B6
:100830000313A100831203133D0883120313A200C4
:10084000831203133E0883120313A300200821041C
:1008500022042304031D4C2C831203133F0883122C
:100860000313A00083120313400883120313A10093
:1008700083120313410883120313A200831203138C
:10088000420883120313A3002008FD002108FE0084
:100890002208FF002308F52E831203133F0883125A
:1008A0000313A00083120313400883120313A10053
:1008B00083120313410883120313A200831203134C
:1008C000420883120313A3002008210422042304F6
:1008D000031D8A2C831203133B0883120313A00009
:1008E000831203133C0883120313A1008312031322
:1008F0003D0883120313A200831203133E088312E0
:100900000313A3002008FD002108FE002208FF00B9
:100910002308F52E831203133B0883120313A00050
:10092000831203133C0883120313A10083120313E1
:100930003D0883120313A200831203133E0883129F
:100940000313A300220D230DA000A400A501A50DF3
:10095000A601A701A101A201A3012008A400003063
:10096000A500831203133F0883120313A000831210
:100970000313400883120313A100831203134108D9
:1009800083120313A200831203134208831203137A
:10099000A300220D230DA000A600A701A70DAC0106
:1009A000AD01A101A201A3010030A7001930260763
:1009B000A000A101A10D2708A1072108803EAE00DB
:1009C0002508803E2E02031DE72C24082002031870
:1009D000092D831203133B0883120313A000831213
:1009E00003133C0883120313A100831203133D0871
:1009F00083120313AC00831203133E088312031304
:100A0000AD002008FD002108FE002C08FF002D0885
:100A1000F52E1930831203132407A000A101A10DA4
:100A20002508A1072108803EAE002708803E2E023F
:100A3000031D1C2D2608200203183E2D83120313CC
:100A40003F0883120313A00083120313400883128C
:100A50000313A10083120313410883120313AC0094
:100A600083120313420883120313AD002008FD0014
:100A70002108FE002C08FF002D08F52E8312031319
:100A80003B0883120313A000831203133C08831254
:100A90000313A100831203133D0883120313AC0058
:100AA000831203133E0883120313AD00AC13AD0190
:100AB000AC17831203133F0883120313AE00831293
:100AC0000313400883120313AF008312031341087A
:100AD00083120313B000831203134208831203131B
:100AE000B100B013B101B017831203133B08831296
:100AF0000313B200831203133C0883120313B300E1
:100B0000831203133D0883120313B40083120313EB
:100B10003E0883120313B500350DB601B60DB701BB
:100B2000B801B901361C9F2DA009A109AC09AD0976
:100B3000A00A0319A10A0319AC0A0319AD0A83120A
:100B400003133F0883120313B200831203134008F8
:100B500083120313B3008312031341088312031398
:100B6000B40083120313420883120313B500350D3A
:100B7000B601B60DB701B801B901361CCA2DAE09D0
:100B8000AF09B009B109AE0A0319AF0A0319B00AD7
:100B90000319B10A831203132708803EBA002508FF
:100BA000803E3A02031DD62D240826020318FD2D8F
:100BB0008312031326082402B2002708031C270A05
:100BC0002502B3003208B21BF22D003C0319FC2DA4
:100BD00083120313B10CB00CAF0CAE0C013E031C1E
:100BE000E82DFC2D031083120313AE0DAF0DB00DD5
:100BF000B10D013E031CF32D272E8312031324088D
:100C00002602B2002508031C250A2702B300320879
:100C1000B21B172E003C0319212E83120313AD0CB7
:100C2000AC0CA10CA00C013E031C0D2E212E0310B8
:100C300083120313A00DA10DAC0DAD0D013E031CDD
:100C4000182E831203132608A4002708A500831278
:100C500003132E08A0072F0803182F0FA107300831
:100C60000318300FAC0731080318310FAD07200807
:100C7000A6002108A7002C08AE002D08AF00031421
:100C8000AF1F0310031C552EA009A109AC09AD0923
:100C9000A00A0319A10A0319AC0A0319AD0AA80195
:100CA000A901AA018030AB00652E8312031320082E
:100CB00021042C042D04031D652E0030FD0000309E
:100CC000FE000030FF000030F52E003083120313C9
:100CD0002D02031D752E80302C02031D752E003051
:100CE0002102031D752E003020020318832E0310ED
:100CF00083120313A00DA10DAC0DAD0DFF30A407A1
:100D0000031CA503652E83120313A6012D08AF0053
:100D100003199F2E201C942E0230A0070318A10A4D
:100D20000319AC0A0319AD0A031083120313AD0CA7
:100D3000AC0CA10CA00CA40A0319A50A832E8312E3
:100D40000313AC132408A6002508A7000030A71B36
:100D5000FF30AF00AE00270C260CB100B001B00C84
:100D6000A501A4010030A8040030A9043008AA0499
:100D70003108AB042808A0042908A1042A08AC04FF
:100D80002B08AD04200883120313BB008312031346
:100D9000210883120313BC00831203132C0883124F
:100DA0000313BD00831203132D0883120313BE0027
:100DB0003B0883120313A000831203133C08831221
:100DC0000313A100831203133D0883120313A4002D
:100DD000831203133E0883120313A5002008FD00AD
:100DE0002108FE002408FF002508080083120317CD
:100DF00093007F0892007E0891007D0883120317FC
:100E000099008312031790007C0897007B089600D6
:100E10007A0895007908831203179D00831203173F
:100E200094001108831203179A0083120317120803
:100E3000831203179B0083120317130883120317EF
:100E40009C00831203171508831203179E00831258
:100E500003171608831203179F008312031717083E
:100E600083120317A00083120317190883120317B4
:100E70009000831203171A0883120317910083123C
:100E800003171B08831203179200831203171C0811
:100E90008312031793000314931F0310031CB52F31
:100EA000831203171D088312031790008312031780
:100EB0001E08831203179100831203171F08831261
:100EC000031792008312031720088312031793005D
:100ED0000314931F0310031CB52F831203171D085F
:100EE000831203179000831203171E08831203173F
:100EF0009100831203171F088312031792008312B5
:100F0000031720088312031793008312031719088D
:100F1000831203179400831203171A08831203170E
:100F20009500831203171B08831203179600831280
:100F300003171C088312031797001308803E9800BC
:100F40001708803E1802031DAF2F16081202031D5A
:100F5000AF2F15081102031DAF2F1408100203183C
:100F6000B32F0130FC2F0030FC2F83120317190818
:100F7000831203179000831203171A0883120317B2
:100F80009100831203171B08831203179200831228
:100F900003171C08831203179300831203171D08FD
:100FA000831203179400831203171E08831203177A
:100FB0009500831203171F088312031796008312EC
:100FC000031720088312031797001308803E980028
:100FD0001708803E1802031DF72F16081202031D82
:100FE000F72F15081102031DF72F1408100203181C
:0E0FF000FB2F0130FC2F003008003C34003491
:1010000083160313860183160317CD01013083165F
:101010000317CF0083120313DB0183120313D801DC
:101020000830831203135802031826285808903EEC
:10103000D90001300318013EDA00590884008313F7
:101040005A188317B7308000D80A10288316031760
:10105000CC0183160317CE01692108008312031304
:10106000D6000130D7005608003C03193D288312F2
:101070000313D70D013E031C3728831203135709AE
:10108000D60083160317CC05080083120313D4007F
:101090000130D5005408003C03195428831203136F
:1010A000D50D013E031C4E288312031355088316E9
:1010B0000317CC04080083160317CC000800831222
:1010C0000313D1007F08D0007E087D08D2005008AD
:1010D000903ED00051080318510F013ED100520834
:1010E000D3005008840083135118831753088000DD
:1010F000080083120313CC007F08CB007E08CE00CB
:101100007D08CD00FF004E089C2083120313CE0003
:101110007F08CD004B08903ECB004C0803184C0FC5
:10112000013ECC004D08CF004B08840083134C18BF
:1011300083174F088000080083120313C6007F083E
:10114000C5000314C61F0310031801294508FF003A
:1011500046088A110A168F238A150A12831203136E
:10116000CA007F08C9007E08C8007D08C700F900D2
:101170004808FA004908FB004A08FC00CD30FD0091
:10118000CC30FE004C30FF003F308A110A12302074
:101190008A150A1283120313CA007F08C9007E0849
:1011A000C8007D08C7000030F9000030FA00903018
:1011B000FB004230FC004708FD004808FE004908DB
:1011C000FF004A088A110A12CD238A150A128312D7
:1011D0000313CA007F08C9007E08C8007D08C70045
:1011E000FD004808FE004908FF004A088A110A1657
:1011F00060228A150A1283120313C8007F08C700F1
:101200005C2983120313450983120313DC00831244
:101210000313460983120313DD00DC0A0319DD0AF8
:101220005C08FF005D088A110A168F238A150A12CE
:1012300083120313CA007F08C9007E08C6007D0818
:10124000C500F9004608FA004908FB004A08FC00FE
:10125000CD30FD00CC30FE004C30FF003F308A1115
:101260000A1230208A150A1283120313E1007F0844
:10127000E0007E08DF007D08DE005E08FD005F08FC
:10128000FE006008FF0061088A110A1660228A15B4
:101290000A1283120313E3007F08E2006208483C4D
:1012A00083120313C700831203136308031C630A2A
:1012B000003C83120313C80083120313C7090314ED
:1012C0004808031C480A003CC8004708FF004808BB
:1012D00008000530831603138100831203130B11DA
:1012E0008B1681010800831203130B118312031361
:1012F0005B08031D8E29831603174F0883160317F7
:101300004C05831203138600EA30810001308312FA
:101310000313DB0083160317CE00E42983120313A3
:101320005B08013A031DAD29831603174D08903E53
:1013300083120313C30001300318013EC4004308A5
:101340008400831344188317000883120313810059
:10135000023083120313DB00E429831203135B08BA
:10136000023A031DE1298312031386018316031732
:101370004D08903E83120313C30001300318013E51
:10138000C400430884008313441883170008523CA8
:1013900083120313810083120313DB0103108316EE
:1013A0000317CF0D83160317CD0A003083160317DA
:1013B0004F04031DE4290130CF0083160317CD012C
:1013C000E42983120313DB010800003400340034E5
:1013D00000347F34F7348E343C344134F2340E34EC
:1013E0003D3446345E3456343D343C34DC348E3443
:1013F0003D34D8347E34B2343D34D3341334D6340F
:101400003D34FB349634F9343D34953482340E3413
:101410003E3430342F3420343E344E34D1343134E1
:101420003E34B234633443343E345C34E6345434B2
:101430003E344B34593466343E34E034B934773476
:101440003E340E34843484343E34B03420348D340D
:101450003E348534B13495343E34DF3437349E34F1
:101460003E341C34B134A6343E343F341D34AF34E2
:101470003E3446347C34B7343E34E234CC34BF346A
:101480003E34C3340D34C8343E343A344034D0345E
:101490003E34A6346134D8343E3408347234E034F7
:1014A0003E3461347134E8343E345F345E34F034B9
:1014B0003E3404343934F8343E34003400340034DB
:1014C0003F34A934D93403343F34D634A8340734F4
:1014D0003F3487346D340B343F34133427340F34A6
:1014E0003F342434D63412343F34683479341634DB
:1014F0003F34E03410341A343F34E5349B341D3427
:101500003F341E341B3421343F34E3348D342434CF
:101510003F348C34F33427343F341B344C342B3475
:101520003F348D3497342E343F343D34D534313408
:101530003F342934053435343F34AB342634383421
:101540003F34C13439343B343F346C343E343E3460
:101550003F34AD34343441343F3433341B344434B9
:101560003F344D34F33446343F340634BB344934CD
:101570003F34AC3473344C343F34EF341B344F3489
:101580003F34D034B33451343F34F7343B345434E3
:101590003F341434B33456343F34CE3419345934D0
:1015A0003F347E346F345B343F342434B4345D34A0
:1015B0003F341934E7345F343F3403340934623440
:1015C0003F343B34193464343F341A3417346634AE
:1015D0003F34EF34033468343F346A34DE346934E2
:1015E0003F34E334A5346B343F34AB345B346D3477
:1015F0003F341934FF346E343F3486348F347034C2
:101600003F3499340D3472343F34AB34783473340E
:101610003F341434D03474343F34233415347634A6
:101620003F343034473477343F349534653478343C
:101630003F345034703479343F340A3468347A3467
:101640003F341B344C347B343F3482341C347C3480
:101650003F344034D9347C343F34563482347D3482
:101660003F34C23417347E343F34DD3498347E3412
:101670003F344F3406347F343F34183460347F3481
:101680003F343734A6347F343F340634D8347F3483
:101690003F342B34F6347F343F340034003480340C
:1016A0003F3483160313C7007F08C6008316031751
:1016B0004E08013A031DFB2BCE01831603174D087C
:1016C00083160313C8000230FF0048088A110A1667
:1016D000B7238A150A1283160313C900E03ECA0015
:1016E00000300318013ECB004A08840083134B18D6
:1016F00083170008CC00840A0008CD004908213E69
:10170000C90001300318013ECA0049088400831350
:101710004A1883170008CB00840A0008CE004B0843
:1017200083160317490783160313C900831603178B
:101730004A0883160313CA004E0803184E0FCA073F
:101740004908FD004A08FE004C08FF004D088A15B4
:101750000A1291248A150A1283160313CA007F08FD
:10176000C900FF004A088A150A129C208A150A122D
:1017700083160313CA007F08C900CB004808903EB7
:10178000C90001300318013ECA00490884008313D0
:101790004A1883174B0880004808031DFB2B460896
:1017A00083160317C9078316031347080318470A4C
:1017B0000319DD2B83160317CA07031483160317B7
:1017C000CA1F0310031CE82B6730C9000130CA0090
:1017D0006830FD000130FE00831603174908FF0042
:1017E0004A088A110A1692208A150A1283160317CC
:1017F000CA007F08C900080083160313BC007F08D5
:10180000BB007E08BE007D08BD007C08C0007B08D0
:10181000BF00C1013F084004031D122C83160317AB
:10182000C901CA01013083160313BF0009308316B2
:1018300003133F020318882C3F085B3EC0000130B1
:101840000318013EC2004008840083134218831726
:101850000008C30043080319842CC3030230FF00AF
:1018600043088A110A16B7238A150A12831603132E
:10187000C000E03EC20000300318013EC400420830
:1018800084008313441883173B088000840A3C08B3
:10189000800084034008213EC00001300318013E4F
:1018A000C2003F08C400C501FF30C407031CC503C4
:1018B0003D08FD003E08FE004408FF0045088A116F
:1018C0000A16F2228A150A1283160313C5007F082E
:1018D000C400400884008313421883174408800022
:1018E000840A4508800084030130C0004308003C9E
:1018F0000319802C83160313C00D013E031C7A2CA0
:10190000831603134008C10483160313BF0A162C61
:101910008316031341088A150A125B208A150A12DE
:10192000080083120317C2007F08C1007E08C400AC
:101930007D08C3000130C500C6010314C41F031095
:101940000318A62C0130C700C801B02CFF30831249
:101950000317C700C800C309C409C30A0319C40A8E
:101960006830FD000130FE00831203174308FF00BA
:1019700044088A110A1692208A150A128312031744
:10198000C4007F08C3004408803E803E031DCA2C6B
:101990005B304302031CE12C831203174408803E92
:1019A000803E031DD52CB53043020318E12C831271
:1019B00003174308B43CC3004408031C440A003C1A
:1019C000C400831203174408803E803E031DEA2CA6
:1019D000B5304302031C002D831203174408803ED8
:1019E0007F3E031DF52C0F3043020318002D4C30B1
:1019F00083120317C307031CC403FF30C500C600CE
:101A0000831203174408803E7F3E031D092D0F30CB
:101A10004302031C232D831203174408803E7F3E9C
:101A2000031D142D693043020318232D831203175D
:101A30004308683CC3004408031C440A013CC4003A
:101A4000FF30C500C600831203174308FD00440899
:101A5000FE000430FF0000308A110A16F2228A15B7
:101A60000A1283120317C4007F08C300E53EC300B7
:101A700044080318440F093EC4004308FE0044080C
:101A8000FF0080308A110A1698218A150A128312E3
:101A90000317CC007F08CB007E08CA007D08C90070
:101AA0004108FF0042088A110A168F238A150A127C
:101AB00083120317C4007F08C3007E08C2007D089C
:101AC000C1004908F9004A08FA004B08FB004C081D
:101AD000FC004108FD004208FE004308FF004408E6
:101AE0008A110A1230208A150A1283120317C400C1
:101AF0007F08C3007E08C2007D08C100FD004208C7
:101B0000FE004308FF0044088A110A1660228A1565
:101B10000A1283120317CE007F08CD008312031729
:101B20004508FD004608FE004708FF0048088A11E6
:101B30000A16F2228A150A1283120317C2007F08BE
:101B4000C100831203174D08FD004E08FE008312EA
:101B500003174108FF0042088A110A16F2228A156B
:101B60000A1283120317C2007F08C100FF00420857
:101B7000080083120317D2007F08D1007E08D0002E
:101B80007D08CF0083120317D70083120317500874
:101B900083120317D8008312031751088312031707
:101BA000D90083120317520883120317DA0057086B
:101BB00083120317CF0083120317580883120317E9
:101BC000D00083120317590883120317D100831220
:101BD00003175A0883120317D2004F085004510408
:101BE00052040319132E8312031757088312031785
:101BF000CF0083120317580883120317D0008312F3
:101C00000317590883120317D100831203175A08C8
:101C100083120317D200520DD301D30DD401D50185
:101C2000D601531C1B2E0030FD000030FE0000309A
:101C3000FF000030932E83120317570883120317F7
:101C4000CF0083120317580883120317D0008312A2
:101C50000317590883120317D100831203175A0878
:101C600083120317D200510D520DCF00D300D401BF
:101C7000D40DD501D601D001D101D2016A30CF07F0
:101C8000FF30031CD007FF30031CD107FF30031CBB
:101C9000D2074F08D3005008D40083120317570807
:101CA00083120317CF0083120317580883120317F8
:101CB000D00083120317590883120317D10083122F
:101CC00003175A0883120317D200D113D201D11778
:101CD000D309D409D30A0319D40A5308D31B802E7D
:101CE000003C03198A2E031083120317D21B03141E
:101CF000D20CD10CD00CCF0C013E031C732E8A2EBB
:101D0000031083120317CF0DD00DD10DD20D013E5C
:101D1000031C812E831203174F08FD005008FE009C
:101D20005108FF005208080083120317B4007F080F
:101D3000B3007E08B2007D08B100320433043404DD
:101D4000031DAA2E0030FD000030FE000030FF0011
:101D50000030632F963083120317B500B60183124B
:101D600003173408FF390319BE2E0310B40CB30C4B
:101D7000B20CB10CB50A0319B60AAF2E83120317C1
:101D80003508B7003608B80000303402031DD22EE3
:101D900080303302031DD22E00303202031DD22EBA
:101DA000003031020318F52E031083120317B10D12
:101DB000B20DB30DB40DFF30B507031CB6030030F0
:101DC0003402031DED2E80303302031DED2E003052
:101DD0003202031DED2E00303102031CD42E83127B
:101DE00003173508B7003608B80083120317320806
:101DF000B6007F303305B900BA013108B500FF3AAB
:101E0000031D152F3608FF3A031D152F39087F3A99
:101E1000031D152F3A08003A031D152FB101B20119
:101E2000B301B401B70A0319B80A83120317B31335
:101E30003708B5003808B6000030B61BFF30BA00CE
:101E4000B900360C350CBC00BB01BB0CB801B701A6
:101E50000030B1040030B2043B08B3043C08B404C1
:101E6000310883120317BD0083120317320883124F
:101E70000317BE0083120317330883120317BF0032
:101E800083120317340883120317C0003D0883121E
:101E90000317B100831203173E0883120317B20021
:101EA000831203173F0883120317B300831203172B
:101EB000400883120317B4003108FD003208FE0009
:101EC0003308FF00340808003030FE001330FF00F4
:101ED00080308A110A16E6218A150A12831203132A
:101EE000E5007F08E4003230E6001330E70083129B
:101EF00003136408E8006508E900FF30E407031CE9
:101F0000E503680869040319F42F04306607E80044
:101F1000E901E90D6708E9076808FE006908FF00A4
:101F200080308A110A16E6218A150A1283120313D9
:101F3000EB007F08EA006608FE006708FF008030BB
:101F40008A110A16E6218A150A1283120313ED007C
:101F5000E9007F08EC00E80002306607E800E901CC
:101F6000E90D6708E9076808FE006908FF0080308E
:101F70008A110A16E6218A150A1283120313E90050
:101F8000EF007F08E800EE00831203136A08EE00FA
:101F90006B08EF00FF30EA07031CEB036E086F04C9
:101FA0000319ED2F6C08FE006D08FF0080308A11C8
:101FB0000A16D3218A150A1283120313EE00680849
:101FC00084008313691883176E088000EC0A0319D4
:101FD000ED0AE80A0319E90AC42F06308312031335
:101FE000E6070318E70A772F8A110A16622B080002
:0E1FF000083400348834FF34003400340034E8
:1020000083160313D2007F08D1007E08D0007D081C
:10201000CF007C08D6007B08D5007A08D400790868
:10202000D300D701D801D901DA010830DB008316CB
:1020300003134F1C29285308D70754080318540FBB
:10204000D80755080318550FD90756080318560F17
:10205000DA0783160313501C41285508DF00540883
:10206000DE00DC010030D7075308DD0003185D0FE8
:10207000D8075E0803185E0FD9075F0803185F0FC3
:10208000DA0783160313511C59285408DF0053083C
:10209000DE00DD01DC010030D707003003185D0FE2
:1020A000D8075E0803185E0FD9075F0803185F0F93
:1020B000DA0783160313521C70285308DF00DE0171
:1020C000DD01DC010030D707003003185D0FD807B1
:1020D0005E0803185E0FD9075F0803185F0FDA0761
:1020E000831603134F08DC005008DD005108DE00A2
:1020F0005208DF0003105F0CD2005E0CD1005D0CB3
:10210000D0005C0CCF000310D30DD40DD50DD60D2F
:10211000DB0B17285708FD005808FE005908FF0080
:102120005A08080083160317A1007F08A0007E0844
:10213000A3007D08A2000314A11F0310031CE428C0
:102140000314A31F0310031CC7282009A40021099E
:10215000A500A40A0319A50A2209A6002309A700BD
:10216000A60A0319A70A2608FD002708FE0024086E
:10217000FF0025088A110A16AF228A110A16831653
:102180000317A5007F08A400FF0025081B2983165C
:1021900003172009A4002109A500A40A0319A50A10
:1021A0002208FD002308FE002408FF0025088A11EC
:1021B0000A16AF228A110A1683160317A5007F0894
:1021C000A400FF0025081B29031483160317A31F6F
:1021D0000310031C06292209A4002309A500A40A50
:1021E0000319A50A2408FD002508FE002008FF00A9
:1021F00021088A110A16AF228A110A1683160317BC
:10220000A5007F08A400FF0025081B2983160317DB
:102210002208FD002308FE002008FF0021088A1183
:102220000A16AF228A110A1683160317A1007F0827
:10223000A000FF0021080800831603179B007F08F9
:102240009A007E0899007D08980019041A041B045E
:10225000031D32290030FD000030FE000030FF0079
:10226000003097290030F9000030FA000030FB0000
:102270000030FC00831603171808FD001908FE0043
:102280001A08FF001B088A110A12F6268A110A167C
:10229000831603179C001C0803197A299F009C00D1
:1022A0009D009E001C08FD001D08FE001E08FF008A
:1022B0001F088A150A12B9258A110A1683160317F0
:1022C0009F007F089E007E089D007D089C009C0961
:1022D0009D099E099F099C0A03199D0A03199E0ADC
:1022E00003199F0A1C08FD001D08FE001E08FF00C0
:1022F0001F089729831603171808FD001908FE0008
:102300001A08FF001B088A150A12B9258A110A1635
:10231000831603179B007F089A007E0899007D08AA
:102320009800FD001908FE001A08FF001B080800AD
:10233000003A0319A229803A0319B229FD01FE01CE
:10234000FF0100347E08840083137F188317000880
:10235000FD00840A0008FE00840A0008FF00840AC9
:10236000000808008A110A16E121FD00FE0FFF0394
:10237000FF0A8A110A16E121FC00FE0FFF03FF0A83
:102380008A110A16E121FB00FE0FFF03FF0A8A11E2
:102390000A16E121FA007D08FD007C08FE007B089A
:1023A000FF007A080800003A0319DA29803A031975
:1023B000E12900347E08840083137F188317000806
:1023C00008007F088A007E0882000800003A03198E
:1023D000EE29803A0319F829FF0100347E088400B1
:1023E00083137F1883170008FF00840A0008080081
:1023F0008A110A16E121FD00FE0FFF03FF0A8A1170
:102400000A16E121FC007D08FF007C080800831605
:102410000317AB007F08AA007E08A9007D08A8006A
:102420000314AB1F0310031C422A2809AC0029091E
:10243000AD002A09AE002B09AF00AC0A0319AD0AA2
:102440000319AE0A0319AF0A2C08FD002D08FE007F
:102450002E08FF002F088A150A1294268A110A16E0
:1024600083160317AF007F08AE007E08AD007D081D
:10247000AC00AF002C08FD002D08FE002E08FF0068
:102480002F085F2A831603172808FD002908FE007D
:102490002A08FF002B088A150A1294268A110A16A8
:1024A00083160317AB007F08AA007E08A9007D08E9
:1024B000A800FD002908FE002A08FF002B080800DC
:1024C00083160317C4007F08C3007E08C2007D087E
:1024D000C100FD004208FE004308FF0044088A11C5
:1024E0000A161C218A110A1683160317C4007F08D6
:1024F000C3007E08C2007D08C1004408803E803EC3
:10250000031D8C2A00304302031D8C2A7F304202B7
:10251000031D8C2AFF304102031C922AFF30FF006A
:102520007F30AE2A831603174408803E813E031D88
:10253000A32AFF304302031DA32A80304202031D59
:10254000A32A013041020318A92A0030FF0080307D
:10255000AE2A831603174108FF00420808008316BD
:102560000317B7007F08B6007E08B9007D08B800E1
:102570003904031DBF2AFF30FF00FF30F12A01306C
:1025800083160317BA008316031738083908BB00EF
:10259000BB1BCF2A0310B80DB90DBA0AC32A0030ED
:1025A000831603173A040319EC2A39083702031D6E
:1025B000DB2A38083602031CE52A8316031738087D
:1025C000B6023908031C390FB7020310831603172C
:1025D000B90CB80CBA03CF2A831603173608FF00CC
:1025E0003708080083120317E5007F08E4007E081F
:1025F000E7007D08E600E801E9010830EA008312FF
:102600000317641C092B6608E80767080318670F9F
:10261000E907831203176408EB006508EC0000303B
:10262000EC1BFF306C1C1C2BEB010030E80766082C
:10263000EC0003186C0FE907831203176408EB0022
:102640006508EC0003106C0CE5006B0CE400031053
:10265000E60DE70DEA0BFF2A6808FF00690808008D
:1026600008340034F43413345B3401340934003456
:10267000FD3407346D34013402340034F8340F343F
:10268000C534013402340034FA340F34C734013411
:1026900002340034D4341334E034003410340034C1
:1026A000E43413342134013410340034FC340F3456
:1026B000C934013402340034FE340F34D1340134CF
:1026C000013400348A150A1200208A110A160030DB
:1026D000FB000030FC00831603174708FD00480884
:1026E000FE00831203176D08FF006E088A150A1298
:1026F000FC238A110A16831203138B1706308316E4
:1027000003139F000514831603174508FF004608AE
:102710008A150A1251238A110A16832B0800831680
:102720000317B300B1007F08B000B2000030B31B44
:10273000FF30B500B4003208FD003308FE00340855
:10274000FF0035088A110A1607228A110A16831615
:102750000317B3007F08B2007E08B1007D08B00007
:10276000FD003108FE003208FF0033080800831620
:102770000317BC007F08BD00BE010830BF008316F0
:1027800003173C1CC52B3D08BE07831603173C08E6
:10279000C0000310400CBC0003103D0DC000BD0084
:1027A000BF0BBF2B3E080800003400340034003457
:1027B0000034003400340034003400340034003479
:1027C0000034003400340034003400340034003469
:1027D0000034003400340034003400340034003459
:1027E000003400340034003400340234043406343D
:0A27F00008340034003400340034D3
:00000001FF
